:100000007228A2008316851283120930A300031000
:100010001020A20CA30B08280314102003146D2831
:100020000318152800008516172885121728003098
:10003000A1005B304028B4002E20200821040319C1
:100040006D28672084133408800664002728282838
:10005000A00A0319A10F252880066D28FF3A8417EE
:1000600080056D28A301A200FF30A207031CA3078F
:10007000031C6D280330A100DF3040203428A1018B
:10008000E83EA000A109FC30031C4928A007031882
:100090004628A0076400A10F462820184F28A01C5E
:1000A0005328000053280800A20001305728A80058
:1000B00023082102031D5E282208200204300318B1
:1000C0000130031902302805031DFF306D28A009F7
:1000D000A109A00A0319A10A0800831303138312BC
:1000E0006400080083169F0183120730990083166D
:1000F0000830850083128501643032200511831693
:1001000005118312B801B9013808A0003908A1000F
:10011000A301FF305420031DB228E830A0000330B3
:10012000A1000530840010301B2032303220E8302E
:10013000A0000330A1000530840010301B2083167E
:1001400010088312012038088316900004308312AF
:10015000850683160511643083123220B80A03190C
:10016000B90F84288228E830A0000330A1000530B0
:10017000840010301B209630322083161008831222
:10018000012052300120553001204930012020301B
:100190000120433001204130012042300120523003
:1001A0000120413001204C300120B3286300D628C3
:02400E00D43F9D
:00000001FF
